:1000000000308A00F6280000FF00030E8301A100E3
:100010007F08A0000A08A8008A01A00E0408A20018
:100020007708A3007808A4007908A5007A08A6003C
:100030007B08A700831383128C308400001C2228C5
:100040000C1839288B1E26280B193B2822088400FF
:100050002308F7002408F8002508F9002608FA000C
:100060002708FB0028088A00210E8300FF0E7F0E60
:1000700009008A114E288A113D28C708031D44280B
:1000800081010130C7004B28A1308100C701FA303F
:100090008F008E0110140B118A112628481C52283B
:1000A00005145328051048080C3C03185E2810104E
:1000B000C8012930C9003630CA0077284A088400B0
:1000C0000008DA004A08840000088E075A080E0269
:1000D0000318702849088400013000078F0774282E
:1000E0004908840000088F07C80AC90ACA0A0C1008
:1000F0008A1126281030D900F701FA01D60CD50C48
:10010000031C88285708F7070318FA0A5808FA0743
:10011000FA0CF70CF90CF80CD90B7E288A119828E8
:100120005208D6005108D500D8010530D7007A28EA
:100130007908D6000310790CFA00780CF900FF3A20
:10014000D300FF307A06D4002930500784005408C9
:10015000FA018000363050078400FA01530880000D
:1001600000344308003A0319B928013A0319C52895
:10017000CC284D08053C031CC0284D08C400F328BA
:1001800024300C1EC1289900F428C6014D08C50072
:100190004508C600C501F3284D08C5044608003CC3
:1001A0000318F128FF3A031DD92845088F3C03188E
:1001B000F1284608063C031CF128031DE3284508E6
:1001C000403C031CF1280310440D013ECF00D00039
:1001D0004608D2004508D100902021300C1EEE28A0
:1001E0009900C301F428C30A8A11362984011F30FB
:1001F0008305813083169900263098009030831251
:10020000980007309F00C301C401C501C601C701A2
:10021000C8012930C9003630CA0000306500831695
:100220000108C0390738810083128F010F088E0042
:1002300010309000CB014B080C3C031C28294B08C4
:10024000D0000130D2009030D1009020CB0A1B2981
:100250008B1683160C14C03083128B04A0308100DF
:100260008C1E30291A08CC00CD00B128302963003B
:02400E006A3F07
:00000001FF
